:1007E00000930000000300000DFE00000000000068
:1007F00000000000000000000000000000000000F9
:100800000234EE009600960701F40002342B023EFB
:10081000420000020826D2AF320000020816D2AF12
:10082000320000022859D2AF32000002081E208A8E
:1008300003020E34900180E06003020E349001ED5B
:10084000E07002A3E06003020E349001EBE070025E
:10085000A3E06003020E3490016DE07002A3E0603B
:1008600003020E349000F1E064206003020E349025
:10087000013FE0FF6003020E34EF704B900117E080
:10088000FBA3E0FAA3E0F91214FDFFAEF09001051E
:10089000E0FBA3E0FAA3E0F91214FDD39FE5F09E7C
:1008A0004003020E347E007F0C7D007B017A0179CB
:1008B00040121740E4900179F0A3F09001F3F0A307
:1008C000F09001F1F0A3F0E4F5B290017DE0FFA318
:1008D000E0900210CFF0A3EFF0C20B300403020D42
:1008E000FF758D20438D20758D8043A808D2AF758C
:1008F0008B02758EC820042E9000F1E064207026D3
:10090000200923E5DB5404701D758A84200913E552
:10091000DB5404700DF586758703000000758601B1
:100920008006D20B8002D20B758B01758A1053A8FA
:10093000F7D39001ECE094909001EBE09401400E2D
:10094000A3E02470F09001EBE034FEF08007E49027
:1009500001EBF0A3F0D39001F8E094909001F7E060
:100960009401400EA3E02470F09001F7E034FEF013
:100970008007E49001F7F0A3F0E4900214F0A3F0F4
:100980001222B2900163EEF0A3EFF0900167EEF057
:10099000A3EFF0C3900211E09FFF900210E09EFED3
:1009A000123E6A900212EEF0A3EFF0D39414EE948C
:1009B00000502E900215E004F07006900214E0043E
:1009C000F0D3900215E09405900214E094004002E8
:1009D000D20BD3900213E0940F900212E0940050D7
:1009E0009FC3900213E09414900212E0940040031D
:1009F000020DE2300B03020DE2900157E0FEA3E08E
:100A0000FF900167E0FCA3E0FD9FEC9E4053ED9F4B
:100A1000FFEC9EFE7C007D031217139001A91216B5
:100A2000D6E47FB87E88FDFC9001A9E0F8A3E0F948
:100A3000A3E0FAA3E0FBD31216B29001A9400A1278
:100A400016E20000EA60020ACAE0FCA3E0FDA3E0AF
:100A5000FEA3E024A8FFEE3461FEE43DFDE43C800B
:100A600062900167E0FEA3E0FFC3900158E09FFFA2
:100A7000900157E09EFE7C007D031217139001A9A0
:100A80001216D6E47FA87E61FDFC9001A9E0F8A3D0
:100A9000E0F9A3E0FAA3E0FBD31216B29001A9405B
:100AA000091216E2000000008020E0F8A3E0F9A39C
:100AB000E0FAA3E0FBC374A89BFF74619AFEE4997B
:100AC000FDE498FC9001A91216D69001A9A3A3E019
:100AD000FFA3E09001A7CFF0A3EFF0900210E0FE9B
:100AE000A3E0FF7C007D09121713ECF8EDF9EEFA94
:100AF000EFFB900167E0FEA3E0FFE4FCFDEB2FFFBE
:100B0000EA3EFEED39FDEC38FCE47B0AFAF9F81216
:100B1000160A900210EEF0A3EFF090013FE06003A0
:100B2000020BF7900108E0FBA3E0FAA3E0F912142E
:100B3000FDFFAEF07C007D03121713ECF8EDF9EE2B
:100B4000FAEFFB9001A7E0FEA3E0FFE4FCFDEB2F32
:100B5000FFEA3EFEED39FDEC38FCE47B04FAF9F8DF
:100B600012160A900100EEF0A3EFF0900108E0FBEE
:100B7000A3E0FAA3E0F91214FDFFAEF07C007D03C0
:100B8000121713ECF8EDF9EEFAEFFB900100E0FE1E
:100B9000A3E0FFE4FCFDEB2FFFEA3EFEED39FDECA8
:100BA00038FCE47B04FAF9F812160A900108E0FB1D
:100BB000A3E0FAA3E0F9EE8FF0121560900100E0D7
:100BC000F9A3E0FFA3E0FBA3E0FAA3E0C98FF012D2
:100BD0001560900105E0FBA3E0FAA3E0F9E4F5F06D
:100BE00012156090010EE0FBA3E0FAA3E0F9E4F532
:100BF000F0121560020DE2900100E0FEA3E0FF7C20
:100C0000007D03121713ECF8EDF9EEFAEFFB9001FB
:100C1000A7E0FEA3E0FFE4FCFDEB2FFFEA3EFEEDC4
:100C200039FDEC38FCE47B04FAF9F812160A90015D
:100C300000EEF0A3EFF0A3E0FBA3E0FAA3E0F9EEEF
:100C40008FF0121560900108E0FBA3E0FAA3E0F931
:100C50001214FDFFD39001A8E09F9001A7E095F04A
:100C60005003020DFF1214FDFFAEF0900102E0FBF5
:100C7000A3E0FAA3E0F91214FDC39FFFE5F09EFE86
:100C8000C3EF9513EE95125003020DFF900105E09E
:100C9000FBA3E0FAA3E0F91214FDFFAEF07C007DA7
:100CA00002121713ECC0E0EDC0E0EEC0E0EFC0E0D0
:100CB000900108E0FBA3E0FAA3E0F91214FDFFAEF7
:100CC000F0900102E0FBA3E0FAA3E0F91214FDC3E7
:100CD0009FFFE5F09EFEE4FCFDD0E0FBD0E0FAD003
:100CE000E0F9D0E0F8EB2FFFEA3EFEED39FDEC38FD
:100CF000FCE47B03FAF9F812160A900105E0FBA365
:100D0000E0FAA3E0F9EE8FF0121560900105E0FB28
:100D1000A3E0FAA3E0F91214FDD39430E5F0947542
:100D20004008747575F030121560900180E0700312
:100D3000020DE2900184E0FEA3E0FFD39400EE9464
:100D4000005003020DE2900105E0FBA3E0FAA3E0EE
:100D5000F91214FDC39FFFE5F09EFE123E6A90015A
:100D6000ADEEF0A3EFF0900105E0FBA3E0FAA3E005
:100D7000F91214FDFFC3900185E09F900184E09576
:100D8000F050209001AEE0940A9001ADE094004054
:100D900012900108E0FBA3E0FAA3E0F9E475F00784
:100DA000121528900105E0FBA3E0FAA3E0F9121464
:100DB000FDFFD3900185E09F900184E095F04022F3
:100DC000D39001AEE0940A9001ADE09400401390FE
:100DD0000108E0FBA3E0FAA3E0F974FF75F0F91253
:100DE0001528200B1AC3900213E09414900212E00D
:100DF0009400500B9000F1E0642070030208DB9037
:100E0000017FE004F09001881216E200000000E487
:100E100090018CF0A3F0A3F0A3F09001D21216E29F
:100E2000000000009001E01216E200000000123EF7
:100E300042123C88229001A9EFF0A3ECF0A3EDF060
:100E4000EFC454F0240AF582E43402F583E0FEA3F3
:100E5000E0C39DFFEE9CFE123E6AD3EF9428EE6441
:100E6000809480406C9001A9E0FBC454F02400F50C
:100E700082E43402F5831216E200000000EBC45451
:100E8000F02404F582E43402F583E4F0A3F0900149
:100E9000A9E0FFC454F02408F582E43402F583E4A9
:100EA000F0A3F0EFC454F0240DF582E43402F5838E
:100EB000E4F09001AAE0FEA3E0FF9001A9E0C45491
:100EC000F0240AF582E43402F583EEF0A3EFF0801B
:100ED0006C9001A9E0C454F02406F582E43402F5D4
:100EE00083E0FEA3E0FFD39400EE9400404F900116
:100EF000AAE0FCA3E0FDD3EF9DEE9C40149001A975
:100F0000E0C454F0240DF582E43402F583E044019A
:100F1000F09001A9E0FFC454F02406F582E4340205
:100F2000F583E0FAA3E0C39DEA9C5011EFC454F0AE
:100F3000240DF582E43402F583E04402F09001A927
:100F4000E0C454F02400F582E43402F583C083C089
:100F500082E0F8A3E0F9A3E0FAA3E0FB9001AAE0A5
:100F6000FEA3E0FFE4FCFDEB2FFFEA3EFEED39FDC2
:100F7000EC38FCD082D0831216D69001A9E0FFC4D1
:100F800054F02404F582E43402F583E475F0011290
:100F900014E7EF75F007A42408F582E43408F5831C
:100FA000E493FE740193FF9001A9E0FDC454F02482
:100FB00008F582E43402F583E0FAA3E0C39FEA9ED9
:100FC0005003021280EDC454F02404F582E434028C
:100FD000F583E0FEA3E0FBEEFAE4F9F89001A9E066
:100FE000C454F02400F582E43402F583E0FCA3E06D
:100FF000FDA3E0FEA3E0FF12160A9001AC1216D684
:101000009001ACA3A3E0FEA3E0FF9001A9E0C454CB
:10101000F02406F582E43402F583E0FCA3E0C39FEC
:10102000FFEC9EFE123E6A9001B0EEF0A3EFF0904E
:1010300001A9E0FD75F007A42403F582E43408F566
:1010400083C37401939FE4939E4031EDC454F02414
:1010500006F582E43402F583E0FEA3E04E601D90C5
:1010600001A9E0FBC454F0240EF582E43402F583B8
:10107000E0FEA3E0C394B8EE940B50479001A9E0C2
:10108000FFC454F02406F582E43402F583E0FCA3A7
:10109000E04C7011EFC454F0240EF582E43402F5F4
:1010A00083E4F0A3F09001ACA3A3E0FEA3E0FF90E3
:1010B00001A9E0C454F02406F582E43402F583EE7D
:1010C0000211A3EB60030211A99001B2F09001B0EC
:1010D000E0FEA3E0FFD39450EE94004006A3740812
:1010E000F0803B9001A9E0C454F0240DF582E43473
:1010F00002F583E064036026D3EF943CEE94004055
:10110000089001B27404F08015D39001B1E09428E6
:101110009001B0E0940040069001B27402F090019A
:10112000A9E0C454F02406F582E43402F583E0FE1D
:10113000A3E0FFE4FCFD9001ACE0F8A3E0F9A3E03C
:10114000FAA3E0FBD31216B2401E9001B2E0FF906A
:1011500001A9E0C454F02406F582E43402F583E4E6
:101160008FF01214E7021214D39001B1E094509062
:1011700001B0E0940050030212149001A9E0C4549D
:10118000F02406F582E43402F583C083C082E0FED9
:10119000A3E0FF9001B2E0FDC3EF9DFFEE9400D00D
:1011A00082D083F0A3EFF0806B9001A9E0C454F0EB
:1011B0002406F582E43402F583E0FEA3E0FF4E70DE
:1011C000169001ACE0F8A3E0F9A3E0FAA3E0FFEA8F
:1011D000FEE9FDE8FC80287C007D071217139001D2
:1011E000ACE0F8A3E0F9A3E0FAA3E02FFFEA3EFEAB
:1011F000E93DFDE83CFCE47B08FAF9F812160A9098
:1012000001A9E0C454F02406F582E43402F583EE2B
:10121000F0A3EFF09001A9E0FBC454F02400F582A4
:10122000E43402F5831216E200000000EBC454F02F
:101230002404F582E43402F583E4F0A3F09001A9DC
:10124000E0FFC454F02408F582E43402F583E4F0AE
:10125000A3F0EFC454F0240DF582E43402F583E4E6
:10126000F09001ACA3A3E0FEA3E0FF9001A9E0C4CD
:1012700054F0240AF582E43402F583EEF0A3EFF093
:101280009001A9E0C454F02406F582E43402F58309
:10129000E0FEA3E0FFD39400EE9400500302134B52
:1012A0009001ABE09FFF9001AAE09EFE123E6A9083
:1012B00001A9E075F007A42405F582E43408F5835C
:1012C000D37401939FE4939E402E9001A9E0FFC444
:1012D00054F02406F582E43402F583E0FDA3E090A7
:1012E00001AACDF0A3EDF0EFC454F0240CF582E494
:1012F0003402F583E4F080539001A9E0FF75F00714
:10130000A42407F582E43408F583E493FEEFC45483
:10131000F0240CF582E43402F583E0C39E502C9057
:1013200001A9E0C454F02406F582E43402F583E018
:10133000FDA3E09001AACDF0A3EDF0EFC454F0249A
:101340000CF582E43402F583E004F09001AAE0FE9B
:10135000A3E0FF22E709F608DFFA8046E709F20872
:10136000DFFA803E88828C83E709F0A3DFFA8032BF
:10137000E309F608DFFA8078E309F208DFFA807003
:1013800088828C83E309F0A3DFFA806489828A83F0
:10139000E0A3F608DFFA805889828A83E0A3F20886
:1013A000DFFA804C80D280FA80C680D4806980F2D7
:1013B0008033801080A680EA809A80A880DA80E25C
:1013C00080CA803389828A83ECFAE493A3C8C582F9
:1013D000C8CCC583CCF0A3C8C582C8CCC583CCDF3C
:1013E000E9DEE7800D89828A83E493A3F608DFF9BA
:1013F000ECFAA9F0EDFB2289828A83ECFAE0A3C81B
:10140000C582C8CCC583CCF0A3C8C582C8CCC5836F
:10141000CCDFEADEE880DB89828A83E493A3F208EA
:10142000DFF980CC88F0EF60010E4E60C388F0EDEC
:101430002402B4040050B9F582EB2402B404005035
:10144000AF23234582239013A473EF8DF0A4A8F05B
:10145000CF8CF0A428CE8DF0A42EFE22BC000BBEB3
:101460000029EF8DF084FFADF022E4CCF875F00890
:10147000EF2FFFEE33FEEC33FCEE9DEC984005FCC5
:10148000EE9DFE0FD5F0E9E4CEFD22EDF8F5F0EE8D
:101490008420D21CFEADF075F008EF2FFFED33FD78
:1014A0004007985006D5F0F222C398FD0FD5F0EA18
:1014B00022C2D5EC30E709B2D5E4C39DFDE49CFC23
:1014C000EE30E715B2D5E4C39FFFE49EFE12145C34
:1014D000C3E49DFDE49CFC800312145C30D507C37B
:1014E000E49FFFE49EFE22C5F0F8A3E028F0C5F0DB
:1014F000F8E582158270021583E038F022BB010AFC
:1015000089828A83E0F5F0A3E022500687F009E79C
:101510001922BBFE07E3F5F009E3192289828A83C9
:10152000E493F5F074019322BB010789828A830258
:1015300014E7500B09C5F027F7C5F01937F722BBA0
:10154000FE0D09F8E325F0F3C5F019E338F322F8AE
:1015500089828A8374019325F0C5F0F8E4933822D8
:10156000BB010A89828A83F0E5F0A3F0225006F7D6
:1015700009A7F01922BBFE06F3E5F009F31922E8EA
:101580008FF0A4CC8BF0A42CFCE98EF0A42CFC8A68
:10159000F0EDA42CFCEA8EF0A4CDA8F08BF0A42DE5
:1015A000CC3825F0FDE98FF0A42CCD35F0FCEB8E86
:1015B000F0A4FEA9F0EB8FF0A4CFC5F02ECD39FE3C
:1015C000E43CFCEAA42DCE35F0FDE43CFC2275F0B1
:1015D00008758200EF2FFFEE33FECD33CDCC33CC38
:1015E000C58233C5829BED9AEC99E58298400CF553
:1015F00082EE9BFEED9AFDEC99FC0FD5F0D6E4CE81
:10160000FBE4CDFAE4CCF9A88222B800C1B90059B4
:10161000BA002DEC8BF084CFCECDFCE5F0CBF97881
:1016200018EF2FFFEE33FEED33FDEC33FCEB33FB15
:1016300010D703994004EB99FB0FD8E5E4F9FA229F
:101640007818EF2FFFEE33FEED33FDEC33FCC9339A
:10165000C910D7059BE99A4007EC9BFCE99AF90F62
:10166000D8E0E4C9FAE4CCFB2275F010EF2FFFEECE
:1016700033FEED33FDCC33CCC833C810D7079BEC19
:101680009AE899400AED9BFDEC9AFCE899F80FD591
:10169000F0DAE4CDFBE4CCFAE4C8F922EB9FF5F0F4
:1016A000EA9E42F0E99D42F0EC6480C8648098456F
:1016B000F022EB9FF5F0EA9E42F0E99D42F0E89CB3
:1016C00045F022E8600FECC313FCED13FDEE13FEB2
:1016D000EF13FFD8F122ECF0A3EDF0A3EEF0A3EFAF
:1016E000F022A8828583F0D083D0821216F91216D8
:1016F000F91216F91216F9E473E493A3C583C5F041
:10170000C583C8C582C8F0A3C583C5F0C583C8C555
:1017100082C822EC8EF0A4CCC5F0CCCDF8EFA4CEDC
:10172000C5F02DFDE43CFCE8A42EC8C5F03DFDE469
:101730003CFCEFA4FFE5F028FEE43DFDE43CFC2288
:10174000EF4E6012EF60010EEDBB010B89828A83C0
:10175000F0A3DFFCDEFA2289F05007F709DFFCA9CD
:10176000F022BBFEFCF309DFFCA9F022D39001ECD0
:10177000E094009001EBE094004003021B4A9001CA
:1017800008E0FBA3E0FAA3E0F91214FDFFAEF0902D
:101790000102E0FBA3E0FAA3E0F91214FDFDACF0B6
:1017A000D39FEC9E4054900108E0FBA3E0FAA3E035
:1017B000F91214FDFFC3ED9FFFEC95F0FED3EF94FB
:1017C00030EE9475400C9001A77475F0A37430F05E
:1017D00080211214FDFFAEF0900102E0FBA3E0FABD
:1017E000A3E0F91214FDC39FFFE5F09E9001A7F05E
:1017F000A3EFF0E49001A1021889900102E0FBA39D
:10180000E0FAA3E0F91214FDFFAEF0900108E0FB4E
:10181000A3E0FAA3E0F91214FDFDACF0C39FFFECC6
:101820009EFED3EF9410EE9427400C9001A77427EE
:10183000F0A37410F0801D900102E0FBA3E0FAA376
:10184000E0F91214FDFFC3ED9FFEEC95F09001A7A7
:10185000F0A3CEF09001A7E0FFA3E09001A1CFF0AC
:10186000A3EFF0300018D3E0942C9001A1E0940194
:1018700040139001A37427F0A37410F08007E49044
:1018800001A3F0A3F0E49001A7F0A3F090013FE0E2
:10189000605B9001A7E0FEA3E0FFD39400EE6480BC
:1018A00094804014D3EF9509EE9508400B9001F118
:1018B000E4F0A37464F08027D39001F2E0940090E8
:1018C00001F1E094004018900105E0FBA3E0FAA3C9
:1018D000E0F91214FDFF9001A7E5F0F0A3EFF0D2BC
:1018E000089001F7740FF0A374A0F0800F9001F539
:1018F0007403F0A374E8F0E4FF123C07D39001A84E
:10190000E094009001A7E0648094805003021AF5EF
:10191000E0F9A3E0FF900105E0FBA3E0FAA3E0C932
:101920008FF01215609001A7E0FEA3E0FFEE339563
:10193000E0FDFCE47BB87A88F9F8C312169C500AE3
:101940009001A77488F0A374B8F0D39001F4E094E8
:10195000009001F3E0940050089000F1E0642070E2
:10196000229001A7E0FEA3E0FFC39496EE6480946A
:10197000805010EF9400EE6480948040447C007DA1
:101980000A803330003B90013FE070169001A7E0E1
:10199000FEA3E0FFC39513EE951250257C027DBC9B
:1019A00080149001A7E0FEA3E0FFC39509EE95081F
:1019B000500F7C027DBC1214B19001A7EEF0A3EF92
:1019C000F090013FE07003021A6B9001F5E07002A5
:1019D000A3E070199001A7E0FEA3E0FDEEFCE4FF98
:1019E000120E359001A7EEF0A3EFF0803E9001A714
:1019F000E0FEA3E0FFC3900136E09FFF900135E0D9
:101A00009EFE123E6AD3EF9428EE64809480401BC1
:101A1000D39001F6E094C89001F5E09400400CA347
:101A2000E0249CF09001F5E034FFF0900135E0FEF9
:101A3000A3E0FF7C007D07121713ECF8EDF9EEFA36
:101A4000EFFB9001A7E0FEA3E0FFEE3395E0FDFC85
:101A5000EB2FFFEA3EFEE93DFDE83CFCE47B08FAA3
:101A6000F9F812160A900135EE800B9001A7E0FFFD
:101A7000A3E0900135CFF0A3EFF0900135E0FEA395
:101A8000E0FFD39405EE9400400EEF9410EE940026
:101A900050069001A7EE8016900131E0FEA3E0FF12
:101AA000900136E02FFF900135E03E9001A7F0A3B2
:101AB000EFF0D39001A8E094309001A7E064809407
:101AC000F540077475F0A37430F0E5DB5404707AC8
:101AD0009001A7E0F9A3E0FF90010EE0FBA3E0FA7C
:101AE000A3E0C98FF01215609001A8E024A8FF9030
:101AF00001A7E08042E5DB5404704F900105E0FB54
:101B0000A3E0FAA3E0F9E4F5F0121560900131E0EA
:101B1000F9A3E0FF90010EE0FBA3E0FAA3E0C98F78
:101B2000F012156090010EE0FBA3E0FAA3E0F912B9
:101B300014FD24A8FFE5F03461F990010BE0FBA34C
:101B4000E0FAA3E0C98FF0121560229001BCECF01E
:101B5000A3EDF09001BBEFF075F00EA424D6F58252
:101B6000E43401F583E0704E9001BBE075F00EA403
:101B700024D2F582E43401F583E0FCA3E0FDA3E088
:101B8000FEA3E0FFE4FBFAF9F8C31216B260279057
:101B900001BBE075F00EA424CEF582E43401F58398
:101BA000E0FCA3E0FDA3E0FEA3E0FFE4F8C312160F
:101BB000B26003021CC79001BEA3A3E0FEA3E0FF36
:101BC000C39001BDE09FFF9001BCE09EFE123E6A03
:101BD0009001BBE0FD75F00EA424D7F582E434013A
:101BE000F583EEF0A3EFF0ED75F00EA424D6F582A8
:101BF000E43401F583E06041ED75F005A42479F546
:101C000082E4343EF583E493FE740193FFED75F0B6
:101C10000EA424D7F582E43401F583E0FCA3E0D3DD
:101C20009FEC9E40149001BBE075F00EA424D6F505
:101C300082E43401F5837405F09001BEE0FCA3E07A
:101C4000FDA3E0FEA3E0FF9001BBE0FB75F00EA456
:101C500024D2F582E43401F5831216D6EB75F00E2A
:101C6000A424DAF582E43401F583E0FEA3E0FFE486
:101C7000FCFD9001BEE0F8A3E0F9A3E0FAA3E0FBCD
:101C800012157F9001BBE0FB75F00EA424CEF58207
:101C9000E43401F5831216D6EB75F00EA424D6F5C4
:101CA00082E43401F583E0D3940074809480401181
:101CB000EB75F00EA424D6F582E43401F583E0142C
:101CC000F09001BE021F0F9001BBE0FB75F00EA467
:101CD00024D2F582E43401F583E0FCA3E0FDA3E027
:101CE000FEA3E0FF9001C21216D6EB75F00EA424FD
:101CF000CEF582E43401F583E0FCA3E0FDA3E0FE31
:101D0000A3E0FF9001C61216D69001C6E0FCA3E046
:101D1000FDA3E0FEA3E0FF9001BBE075F00EA4245C
:101D2000D9F582E43401F583E0F9F81216C3EFFB2C
:101D3000EEFAEDF9ECF89001C6E0FCA3E0FDA3E0BB
:101D4000FEA3E0C39BFFEE9AFEED99FDEC98FCA389
:101D50001216D69001C2E0FCA3E0FDA3E0FEA3E0D2
:101D6000FF9001BEE0F8A3E0F9A3E0FAA3E02FFFA3
:101D7000EA3EFEE93DFDE83CFC9001CAE0F8A3E044
:101D8000F9A3E0FAA3E02FFFEA3EFEE93DFDE83CBF
:101D9000FC9001C61216D69001BEE0FCA3E0FDA3A4
:101DA000E0FEA3E0FF9001BBE0FB75F00EA424D29F
:101DB000F582E43401F5831216D69001C6E0FCA347
:101DC000E0FDA3E0FEA3E0FFEB75F00EA424CEF54A
:101DD00082E43401F5831216D69001C6E0FCA3E03C
:101DE000FDA3E0FEA3E0FFECC0E0EDC0E0EEC0E04C
:101DF000EFC0E09001BBE075F00EA424DAF582E4B8
:101E00003401F583E0FEA3E0FBEEFAE4F9F8D0E05C
:101E1000FFD0E0FED0E0FDD0E0FC12160A9001C633
:101E20001216D69001BEA3A3E0FEA3E0FBEEFA904B
:101E300001C6A3A3E0FEA3E0C39BFFEE9AFE123E01
:101E40006A9001BBE0FD75F00EA424D7F582E4345E
:101E500001F583EEF0A3EFF0ED75F005A42477F51E
:101E600082E4343EF583E493FE740193FFED75F054
:101E70000EA424D7F582E43401F583E0FCA3E0D37B
:101E80009FEC9E5003021F0C9001BEE0FCA3E0FDFE
:101E9000A3E0FEA3E0FF9001BBE0FB75F00EA424DD
:101EA000D2F582E43401F5831216D6EB75F00EA458
:101EB00024DAF582E43401F583E0FEA3E0FFE4FCDC
:101EC000FD9001BEE0F8A3E0F9A3E0FAA3E0FB1265
:101ED000157F9001BBE0FB75F00EA424CEF582E4E3
:101EE0003401F5831216D6EB75F00EA424D6F582D4
:101EF000E43401F5837405F09001BEE0FCA3E0FD3D
:101F0000A3E0FEA3E0FF9001C61216D69001C6A37F
:101F1000A3E0FEA3E0FF22D39001ECE09400900147
:101F2000EBE0940040030222B112388B900188E06C
:101F3000F8A3E0F9A3E0FAA3E0FBE8C0E0E9C0E021
:101F4000EAC0E0EBC0E090011DE0FBA3E0FAA3E0F3
:101F5000F91214FDFFE4FCFDD0E0FBD0E0FAD0E084
:101F6000F9D0E0F8EB2FFFEA35F0FEED39FDEC3863
:101F7000FC9001881216D690018DE004F070069056
:101F8000018CE004F0C390018FE0946490018EE036
:101F9000940050030222B1900188E0FCA3E0FDA36D
:101FA000E0FEA3E0FFECC0E0EDC0E0EEC0E0EFC07B
:101FB000E0A3E0FEA3E0FBEEFAE4F9F8D0E0FFD006
:101FC000E0FED0E0FDD0E0FC12160A900188121667
:101FD000D6900188A3A3E0FFA3E0900186CFF0A3F1
:101FE000EFF0A31216E200000000E490018CF0A3D1
:101FF000F0A3F0A3F09001EBE07002A3E060030215
:1020000022B1900190E07002A3E060030222B1903F
:10201000013FE070030220DB900182E0FEA3E0FFBD
:102020004E7034900186E0FDA3E0900182CDF0A3D4
:10203000EDF0900105E0FBA3E0FAA3E0F91214FD36
:10204000FD900184E5F0F0A3EDF09001927403F0AF
:10205000A374E8F00220F4900186E0FCA3E0FDC345
:10206000EF9DFFEE9CFE123E6A90019BE0FBA3E019
:10207000FAA3E0F9EE8FF0121560900180E070375E
:1020800090019BE0FBA3E0FAA3E0F91214FDC394D6
:102090000AE5F09400501A900105E0FBA3E0FAA3D2
:1020A000E0F91214FDFF900184E5F0F0A3EFF08059
:1020B000069001807401F0900186E0FEA3E0FFD35A
:1020C000900183E09F900182E09E4007E4900181AF
:1020D000F080219001817401F08019E4900182F078
:1020E000A3F0A3F0A3F0900180F0900194F0A3F08E
:1020F000A3F0A3F0900180E070030222B19001846C
:10210000E0FEA3E0FFD39400EE940050030222B15E
:10211000900105E0FBA3E0FAA3E0F91214FDC39FD0
:10212000FFE5F09EFE123E6A9001A7EEF0A3EFF0ED
:10213000A3E4F0A374C8F0900105E0FBA3E0FAA3C8
:10214000E0F91214FDD39494E5F09411400A900143
:10215000A97403F0A37420F09001A7E0FFA3E0901E
:10216000019FCFF0A3EFF0900105E0FBA3E0FAA3FD
:10217000E0F91214FDFFAEF0900184E0FCA3E0FD55
:10218000D39FEC9E400FD39001A8E094649001A7E8
:10219000E094005015C3ED9FEC9E50489001A8E0DC
:1021A00094FA9001A7E09400403AE4900180F09006
:1021B0000182F0A3F0900105E0FBA3E0FAA3E0F9AF
:1021C0001214FDFFC3900185E09F900184E095F01B
:1021D0009001905007E4F0A374C8F0227401F0A3BA
:1021E000742CF022900105E0FBA3E0FAA3E0F912C1
:1021F00014FDFFD3900185E09F900184E095F0509D
:1022000003022283D39001A8E0941E9001A7E094DA
:10221000004070900181E0704190019BE0FBA3E0E1
:10222000FAA3E0F91214FDD39420E5F094034002E0
:10223000804EC3900197E0942C900196E094015059
:1022400042900105E0FBA3E0FAA3E0F91214FDC3FC
:102250009490E5F09401402B8026C3900197E09480
:102260002C900196E09401501A900105E0FBA3E048
:10227000FAA3E0F91214FDC39490E5F09401400331
:10228000123ADC900105E0FBA3E0FAA3E0F9121496
:10229000FDFFC3900185E09F900184E095F050110F
:1022A0009001A8E0941E9001A7E094004003123B27
:1022B00029227F01123A35123CFB758A50902E205C
:1022C0007419F0902E20E030E2F9903E89E4937585
:1022D000F002A42400F582E5F0342EF583E0FFA39C
:1022E000E09001B5CFF0A3EFF0902E20E4F0758AD6
:1022F000107F01123D2D90015DE0FEA3E0FF4E70C6
:102300000E9001B5E0FCA3E0FDECFEEDFF801E7C2D
:10231000007D0312144A9001B6E02FFF9001B5E052
:102320003EFE7802EFCEC313CE13D8F9FF90015DC5
:10233000EEF0A3EFF0900159E07002A3E0700F906F
:10234000015DE0FFA3E0900159CFF0A3EFF0900111
:10235000B71216E200002710E4FF123A35E49001AC
:10236000B2F09001B2E0C394027480948040030202
:10237000249FE4FF123CFB758A50902E207419F0C4
:10238000902E20E030E2F9903E88E49375F002A4AC
:102390002400F582E5F0342EF583E0FFA3E0900100
:1023A000B3CFF0A3EFF0902E20E4F0758A10FF1267
:1023B0003D2D9001B3E0FEA3E0FF900169EEF0A394
:1023C000EFF0900159E0FCA3E0FDEF2DFFEE3CFEA5
:1023D00090015DE0FCA3E0FDC3EF9DFFEE9C90014A
:1023E000B3F0A3EFF090015BE0FEA3E0FF4E700EB0
:1023F0009001B3E0FCA3E0FDECFEEDFF801E78024F
:10240000EFC333CE33CED8F9FF9001B4E02FFF9065
:1024100001B3E03EFE7C007D0512145C90015BEE92
:10242000F0A3EFF090015FE07002A3E0700F900165
:102430005BE0FFA3E090015FCFF0A3EFF090015BC2
:10244000E0FEA3E0FFE4FCFD9001BE1216D6900171
:102450005FE0FCA3E0FDE4FF121B4B90015FEEF098
:10246000A3EFF09001B7E0F8A3E0F9A3E0FAA3E04E
:10247000FB90015FE0FEA3E02400FFEE34F0FE33AA
:1024800095E0FDFCEB2FFFEA3EFEE93DFDE83CFC5C
:102490009001B71216D69001B2E004F002236290C8
:1024A0002E23E4F07F507EC3FDFC9001B7E0F8A33B
:1024B000E0F9A3E0FAA3E0FBD312169C400A9001D6
:1024C000B71216E20000C3509001B7E0FCA3E0FD94
:1024D000A3E0FEA3E0FFEC33500A9001B71216E22E
:1024E00000000000900165E0FAA3E0FB4A700C9048
:1024F00001B7A3A3E0FEA3E0FF80347E007F02EBE0
:10250000FDEAFC121713ECF8EDF9EEFAEFFB90017F
:10251000B7E0FCA3E0FDA3E0FEA3E02BFFEA3EFE54
:10252000E93DFDE83CFCE47B03FAF9F812160A9059
:102530000165EEF0A3EFF0900157E07002A3E070A8
:102540000F900165E0FFA3E0900157CFF0A3EFF0FB
:10255000900127E0F8A3E0F9A3E0FAA3E0FB9001E3
:102560005FE0FEA3E0FFE4FCFDEB2FFFEA3EFEEDA3
:1025700039FDEC38FC9001271216D690012CE004AE
:10258000F0700690012BE004F090012BE0FEA3E038
:10259000FFD3940AEE94004031EFFBEEFAE4F9F831
:1025A000900127E0FCA3E0FDA3E0FEA3E0FF1216EC
:1025B0000A900125EEF0A3EFF0E490012BF0A3F0D8
:1025C0009001271216E20000000090012DE0700239
:1025D000A3E07040900125E0FEA3E0FFC3900160FE
:1025E000E09FFF90015FE09EFE123E6A900123EEA5
:1025F000F0A3EFF0D39406EE9400401890012D74F0
:1026000003F0A374E8F0900130E004F0700690014C
:102610002FE004F0900165E0FEA3E0FF229001A707
:102620007403F0A374E8F0D39001A6E09400900145
:10263000A5E094004021900102E0FBA3E0FAA3E0B2
:10264000F91214FDFF900108E0FBA3E0FAA3E0F902
:10265000E5F08FF01215609001EBE07002A3E060EE
:102660000B9001A7E4F0A37464F0800B90001AE0D3
:10267000641170037420F090013FE0600F7E007FD2
:102680000C7D007B017A017940021740900140E007
:10269000F8A3E0F9A3E0FAA3E0FBE8C0E0E9C0E0BA
:1026A000EAC0E0EBC0E0900102E0FBA3E0FAA3E0A7
:1026B000F91214FDFFE4FCFDD0E0FBD0E0FAD0E01D
:1026C000F9D0E0F8EB2FFFEA35F0FEED39FDEC38FC
:1026D000FC9001401216D6900145E004F07006907F
:1026E0000144E004F09001A7E0FEA3E0FFC39001E5
:1026F0004BE09F90014AE09E500302285890014011
:10270000E0FCA3E0FDA3E0FEA3E0FFECC0E0EDC031
:10271000E0EEC0E0EFC0E0A3E0FEA3E0FBEEFAE4F1
:10272000F9F8D0E0FFD0E0FED0E0FDD0E0FC1216DA
:102730000A9001401216D6900108E0FBA3E0FAA32C
:10274000E0F91214FD241EFFE435F0FEE4FCFD90D8
:102750000140E0F8A3E0F9A3E0FAA3E0FBD31216EE
:10276000B2500302281E9001EBE07002A3E0600368
:1027700002281E30080302281E900108E0FBA3E097
:10278000FAA3E0F91214FDFB900140A3A3E0FEA31D
:10279000E0C39BFFEE95F09001A9F0A3EFF090014C
:1027A00047E004F07006900146E004F0D390014742
:1027B000E09401900146E0940040229001A9E0FEDF
:1027C000A3E0FF900149E09F900148E09E500E90E9
:1027D0000147E024FFF0900146E034FFF09001A9AA
:1027E000E0FFA3E0900148CFF0A3EFF0D3900147C2
:1027F000E09405900146E094004046900140A3A378
:10280000E0F9A3E0FF900108E0FBA3E0FAA3E0C930
:102810008FF0121560E4900146F0A3F08023900140
:1028200040A3A3E0F9A3E0FF900108E0FBA3E0FAD6
:10283000A3E0C98FF0121560E4900146F0A3F0C246
:10284000089001401216E200000000E4900144F0FC
:10285000A3F090014AF0A3F022C0E0C083C082C080
:10286000D0D2AFD39001ECE094009001EBE0940063
:10287000400CA3E024FFF09001EBE034FFF0D39094
:1028800001F0E094009001EFE09400400EA3E024FA
:10289000FFF09001EFE034FFF08002D28AD3900184
:1028A000EEE094009001EDE09400400CA3E024FFE2
:1028B000F09001EDE034FFF0C390014BE094E8901C
:1028C000014AE09403500CA3E004F0700690014A22
:1028D000E004F0D39001F2E094009001F1E0940064
:1028E000400CA3E024FFF09001F1E034FFF0D3901E
:1028F00001F4E094009001F3E09400400CA3E02484
:10290000FFF09001F3E034FFF0D39001FAE094007F
:102910009001F9E09400400CA3E024FFF09001F94D
:10292000E034FFF0D39001F6E094009001F5E094DC
:1029300000400CA3E024FFF09001F5E034FFF0D359
:102940009001F8E094009001F7E09400400CA3E0BF
:1029500024FFF09001F7E034FFF0D39001A4E0945D
:10296000009001A3E09400400CA3E024FFF090014C
:10297000A3E034FFF0D39001FCE094009001FBE071
:102980009400400CA3E024FFF09001FBE034FFF042
:10299000C390018FE0946490018EE09400500CA3EA
:1029A000E004F0700690018EE004F0D3900191E015
:1029B0009400900190E09400400CA3E024FFF0907C
:1029C0000190E034FFF0D3900193E09401900192E4
:1029D000E09400400CA3E024FFF0900192E034FF6B
:1029E000F0D390016EE0940190016DE09400400CF2
:1029F000A3E024FFF090016DE034FFF0D39001A636
:102A0000E094009001A5E09400400CA3E024FFF0C6
:102A10009001A5E034FFF0C390020FE094B890025B
:102A20000EE0940B500CA3E004F0700690020EE050
:102A300004F0C3900209E094F4900208E09401507D
:102A40000CA3E004F07006900208E004F0D39001BB
:102A50002EE0940090012DE09400400CA3E024FFB0
:102A6000F090012DE034FFF0D0D0D082D083D0E0C0
:102A700032D39001ECE09F9001EBE09E400AA3E08E
:102A80009FF09001EBE09EF0D39001F0E09F900169
:102A9000EFE09E400CA3E09FF09001EFE09EF080FD
:102AA00002D28AD39001EEE09F9001EDE09E400AB1
:102AB000A3E09FF09001EDE09EF0C390014BE09405
:102AC000E890014AE09403500AA3E02FF090014AF5
:102AD000E03EF0D39001F2E09F9001F1E09E400AC9
:102AE000A3E09FF09001F1E09EF0D39001F4E09F0D
:102AF0009001F3E09E400AA3E09FF09001F3E09E76
:102B0000F0D39001FAE09F9001F9E09E400AA3E023
:102B10009FF09001F9E09EF0D39001F6E09F9001C4
:102B2000F5E09E400AA3E09FF09001F5E09EF0D30F
:102B30009001F8E09F9001F7E09E400AA3E09FF02B
:102B40009001F7E09EF0D39001A4E09F9001A3E0F4
:102B50009E400AA3E09FF09001A3E09EF0D3900175
:102B6000FCE09F9001FBE09E400AA3E09FF09001F3
:102B7000FBE09EF0C390018FE0946490018EE0949E
:102B800000500AA3E02FF090018EE03EF0D39001B8
:102B900091E09F900190E09E400AA3E09FF0900199
:102BA00090E09EF0EF2401FDE43EFCD3900193E021
:102BB0009D900192E09C400AA3E09FF0900192E07A
:102BC0009EF0EF2401FDE43EFCD390016EE09D9069
:102BD000016DE09C400AA3E09FF090016DE09EF043
:102BE000D39001A6E09F9001A5E09E400AA3E09F3C
:102BF000F09001A5E09EF0C390020FE094B890021F
:102C00000EE0940B500AA3E02FF090020EE03EF08D
:102C1000C3900209E094F4900208E09401500AA3E2
:102C2000E02FF0900208E03EF0D390012EE09F905C
:102C3000012DE09E400AA3E09FF090012DE09EF060
:102C4000227E007FFF7D007B017A00790012174011
:102C50007E007FA77D007B017A0179001217407EFC
:102C6000007F147D007B017A0179EA121740902DD4
:102C7000E0E493900001F09000047411F0A374223A
:102C8000F0A37433F0902DE2E493900012F0902DB5
:102C9000E3E493900014F09000FB7401F090003690
:102CA0007410F09000F1F0900024F0A37420F090E4
:102CB00001027401F0A37400F0A37440F0900108C5
:102CC0007401F0A37400F0A37444F0900105740142
:102CD000F0A37400F0A37442F090010B7401F0A310
:102CE0007400F0A3742EF0A37401F0A37400F0A399
:102CF000742AF0A37401F0A37400F0A37428F09078
:102D000001207401F0A37400F0A37460F090011D21
:102D10007401F0A37400F0A37422F090019B74017D
:102D2000F0A37400F0A37480F090013C7401F0A350
:102D30007400F0A37418F09001397401F0A37400CA
:102D4000F0A3741BF09001147401F0A37400F0A3BD
:102D50007432F0A37401F0A37400F0A37426F0A3FE
:102D60007401F0A37400F0A37434F0900114E0FB3C
:102D7000A3E0FAA3E0F9E475F0C81215609001171A
:102D8000E0FBA3E0FAA3E0F9E475F06412156090AB
:102D9000011AE0FBA3E0FAA3E0F9E475F09612153E
:102DA000607512007513C87508007509969001EBDF
:102DB0007407F0A374D0F0E49001EAF0227E007F63
:102DC000047D007B017A01795B1217407E007F044D
:102DD0007D007B017A01795F02174000000000004E
:102DE0000301AB9374AA7583F5758255A574557567
:102DF00083FA7582AAA574A57583F5758255A522F7
:102E000002020AB00BB60CFF090208FF0DF70E0410
:102E1000130714101080019212070D030F0404040D
:102E20000101110808120909030280900179E0FEEE
:102E3000A3E0FFC39404EE9400502F900100E0FC47
:102E4000A3E0FDEF25E0FFEE33FE74712FF58274F1
:102E5000013EF583ECF0A3EDF090017AE004F07010
:102E600006900179E004F0022F329001B47401F071
:102E70009001B4E0FFC3940474809480502AEF253D
:102E8000E02471F582E43401F583E0FCA3E0FDEF7A
:102E900025E0246FF582E43401F583ECF0A3EDF036
:102EA0009001B4E004F080C890013FE060028073BC
:102EB000900102E0FBA3E0FAA3E0F91214FDFF90F9
:102EC0000100E0FCA3E0FDC3EF9DFFE5F09CFE12D6
:102ED0003E6AC3EF9428EE648094805046900108C7
:102EE000E0FBA3E0FAA3E0F91214FDFFC390010197
:102EF000E09FFF900100E095F0FE123E6AC3EF9460
:102F000014EE6480948050059001088003900102C3
:102F1000E0FBA3E0FAA3E0F91214FDFF900177E5CE
:102F2000F0800B900100E0FFA3E0900177CFF0A3C9
:102F3000EFF09001B01216E200000000E49001B43E
:102F4000F09001B4E0FFD390017AE09F900179E026
:102F50009400403D9001B0E0F8A3E0F9A3E0FAA3AB
:102F6000E0FBA3E025E02471F582E43401F583E081
:102F7000FEA3E0FFE4FCFDEB2FFFEA3EFEED39FD92
:102F8000EC38FC9001B01216D69001B4E004F08049
:102F9000B09001B0E0FCA3E0FDA3E0FEA3E0FFECF5
:102FA000C0E0EDC0E0EEC0E0EFC0E0900179E0FEEF
:102FB000A3E0FBEEFAE4F9F8D0E0FFD0E0FED0E0C9
:102FC000FDD0E0FC12160A9001B01216D69001B0A6
:102FD000A3A3E0FEA3E0FF229001AAEFF0902E222F
:102FE000E0FF9001AEE4F0A3EFF0758A50902E223E
:102FF0007401F09001AAE075F002A42410F582E5B6
:10300000F0342EF5837402F0A3E4F09001ABF0905D
:1030100001ABE0FFC3940C74809480400302314202
:10302000EFF87E01E4088006CEA2E713CE13D8F8AD
:10303000FF9001ACEEF0A3EFF04E70079001ACF002
:10304000A304F0902E207419F0902E20E030E2F9C5
:103050009001AAE0FF75F002A42400F582E5F034A7
:103060002EF583E0FCA3E0D394FFEC940740597560
:10307000F002EFA42410F582E5F0342EF583E0FE93
:10308000A3E0FF9001ACE0FCA3E0FDEF2DFFEE3CE0
:10309000FEC3EF94FFEE94039001AAE075F0025096
:1030A00013A42410F582E5F0342EF583EC8DF01294
:1030B00014E7807EA42410F582E5F0342EF58374A5
:1030C00003F0A374FFF0806A9001AAE0FF75F0029C
:1030D000A42410F582E5F0342EF583E0FCA3E0FD96
:1030E0009001ACE0FAA3E0FBD3ED9BEC9A402D7588
:1030F000F002EFA42410F582E5F0342EF583C083AE
:10310000C082C3A3E09BFF0582D58202158315828E
:10311000E09AD082D083F0A3EFF080169001AAE06D
:1031200075F002A42410F582E5F0342EF583E4F066
:10313000A3F0902E20E4F0F58D9001ABE004F002B6
:10314000300F9001AEA3E0902E22F0758A1022E499
:10315000F526F525F524F523F526F525F524F523A3
:10316000F522C3E5229403748094805027E522253C
:10317000E0240AF8E6FE08E6FFE4FCFDE5262FF56C
:1031800026E5253EF525ED3524F524EC3523F523FC
:10319000052280CEE47B03FAF9F8AF26AE25AD24F4
:1031A000AC2312160A90017DEEF0A3EFF0E4752631
:1031B000A8752561F524F523F522C3E5229403744F
:1031C0008094805073E52225E0240AF8E6FE08E6A4
:1031D000FF90017DE0FCA3E0FDC3EF9DFFEE9CFEB0
:1031E000123E6AD3EF940AEE6480948040129001FC
:1031F0007DE0FEA3E0FF900157E0FCA3E0FD801519
:10320000E52225E0240AF8E6FE08E6FF900157E0F3
:10321000FCA3E0FDC3EF9DFFEE9CFE3395E0FDFCBB
:10322000E5262FF526E5253EF525E5243DF524E5A3
:10323000233CF52305228082E47F607EEAFDFCAB1F
:1032400026AA25A924A823D31216B2400BE475267A
:10325000607525EAF524F523AE25AF26221238FF46
:10326000122DBDE4900179F0A3F0900165F0A3F078
:10327000900163F0A3F0900167F0A3F07F03123692
:103280008D900100E0F9A3E0FFA3E0FBA3E0FAA327
:10329000E0C98FF0121560900100E0F9A3E0FF9003
:1032A0000108E0FBA3E0FAA3E0C98FF012156090DB
:1032B0000105E0FBA3E0FAA3E0F9E4F5F0121560E4
:1032C00090010BE0FBA3E0FAA3E0F9746175F0A8AC
:1032D000121560900111E0FBA3E0FAA3E0F974611C
:1032E00075F0A812156090010EE0FBA3E0FAA3E0D0
:1032F000F9E4F5F0121560E4900137F0A3F09001C5
:103300003FF0FE7F1BFD7B017A0179801217407E22
:10331000007F0C7D007B017A017940121740E49018
:1033200001F9F0A3F09001F7F0A3F09000367410CB
:10333000F0E490004BF09001ED7403F0A37420F0E2
:103340009001FDE0700FC39001ECE094F49001EB6C
:10335000E09401500A9001EB7401F0A374F4F022A0
:10336000D39001ECE094009001EBE0940040030264
:10337000342A3000209001A3E07002A3E0600875B9
:10338000121F751340800675121775137075081398
:10339000750988800C7512007513C87508007509C9
:1033A00096900105E0FBA3E0FAA3E0F91214FDFFFB
:1033B000AEF0C39513EE9512500F90013FE0601AE6
:1033C000C3EF9509EE950840119001F3E07002A358
:1033D000E0702E90013F04F080279000F1E064201F
:1033E0009001F37005F0A3F08006E4F0A374C8F038
:1033F000E490013FF09001F1F0A3F09000367410DA
:10340000F090013FE0FF601D900024E06410900008
:103410003670057410F080037420F09001ED740391
:10342000F0A37420F090004BEFF022C0E0C083C006
:1034300082C0D075D018D2AFE5DB30E424D209C207
:1034400006E5DB30E116123E5EF583E0F5DFEF6462
:10345000077067D28A900007F00234DFC205023499
:10346000E2E5DB30E52C9000F0E064AA7017758A85
:1034700010F5DAC2AFF5B2F5A8F5A9F58B758E0196
:10348000758DC080FED204300604C2068054C20985
:103490008050C206E5DB30E123E5DB30E044123E3C
:1034A0005EF583E0F5DFEF24F9600824EE700BD2BF
:1034B0000A8007D28A900007E4F0802320050A786A
:1034C00014A6DFD205D2068019123E5EF583E5DF31
:1034D000F0EF642470099001ED04F0A374F4F07827
:1034E000140675DBFFD0D0D082D083D0E032787F55
:1034F000E4F6D8FD75812602353802000002371047
:10350000E493A3F8E493A34003F68001F208DFF408
:103510008029E493A3F85407240CC8C333C4540F80
:103520004420C8834004F456800146F6DFE4800B53
:103530000102040810204080903D8AE47E019360DF
:10354000BCA3FF543F30E509541FFEE493A3600180
:103550000ECF54C025E060A840B8E493A3FAE493EA
:10356000A3F8E493A3C8C582C8CAC583CAF0A3C898
:10357000C582C8CAC583CADFE9DEE780BE900139CB
:10358000E0FBA3E0FAA3E0F91214FD641045F0702B
:1035900003123A8E900001E064AA70031239D490AD
:1035A0000013E0FF7E0064107002D203EF64204E2F
:1035B0007002C20312379020070890001AE06410CE
:1035C000700E90001A7411F0C2079001EA7401F0B5
:1035D0009000FBE06006E4F09001EAF090016DE0FD
:1035E0007004A3E06401701090016DF0A3F09001ED
:1035F000A5F0A3F09001EAF030040CC2049001EDB4
:103600007401F0A374F4F02290014C7408F0A374D8
:1036100098F0123C487E007F047D007B017A01799E
:10362000571217407F01123E02E4FF123E02902E15
:1036300012E0FEA3E0C39405EE9400400F902E121A
:10364000E0FEA3E0D394F0EE9403400BE490014C31
:10365000F0A3F0FF123E02902E23E4F090001D74C0
:1036600010F0902E12E0FEA3E0FF7C007D0A121401
:103670004A90014DE02FFF90014CE03EF990013C53
:10368000E0FBA3E0FAA3E0C98FF00215609001B05F
:10369000EFF0E4A3F09001B0E0FFA3E0C39F502E51
:1036A0001222B2123DDC900167EEF0A3EFF08E1013
:1036B000F511C8740AC87400FCE4FDFB7A00790CAB
:1036C000FE7F061214249001B1E004F080C712318D
:1036D0004F900100EEF0A3EFF0900165E0FEA3E053
:1036E000FFC3900134E09FFF900133E09EFE123E45
:1036F0006A7C007D051214B1900131ECF0A3EDF06D
:10370000900165E0FFA3E0900133CFF0A3EFF0223A
:1037100053A87F123DB6122C41123E2612080E43CA
:10372000A880E4F58D9000F17420F012357D9001B1
:10373000EAE014601814601A14602D14603F240429
:1037400070E01236089001EA7401F080D512325D03
:103750008023123D5C12380F900025E0641070C287
:103760009001EA7404F080BA12082E9001ED7403FF
:10377000F0A37420F09001EA7402F080A5123BBF20
:10378000900025E06410609A9001EA7401F0809244
:103790009001FEE014602114604324027060300345
:1037A000139001FE7401F0D202D2009001FB04F0EC
:1037B000A37458F0C20180469001FBE07002A3E0C0
:1037C0007002C2022003379001FE7402F0D201C2DF
:1037D00002C2009001FBF0A37458F080219001FB1D
:1037E000E07002A3E070179001FE200303F0800C4C
:1037F0007401F09001FB04F0A37458F0C2012001A1
:103800000330020A900025E064106002D2072230E3
:103810008A789001EBE07002A3E0706E90016DE099
:103820007002A3E07064F5B2758D20438D20758D14
:103830009043A808D2AF758B4090012DE0FEA3E025
:10384000FF4E6005758E148003758E4020042F2076
:10385000092CE5DB54047026758A84200920E5DBF9
:103860005404701AF586758703000000758601EF11
:103870004E60047F2880027F787E00122A71758B4B
:1038800001758A1053A8F7123E4222758D20438D90
:1038900020538D7FE4F5B275B6FF75B7FF75B2A200
:1038A00043B20153A8FB538B7F758B10438B08E504
:1038B0008B20E7030080F8538B7F758B11438B08B7
:1038C000E58B20E7030080F8900219E5B5F0A3E549
:1038D000B4F0758B01E4F5B2123E42E4F58D90022E
:1038E00016E0FBA3E0FAA3E0F91214FDFF90011D1E
:1038F000E0FBA3E0FAA3E0F9E5F08FF00215607EAB
:10390000007F1C7D007B017A0179CE121740E4FD17
:10391000EDC39402748094805057ED75F005A42493
:1039200076F582E4343EF583E493FFED75F00EA462
:1039300024D9F582E43401F583EFF0ED75F00EA49F
:1039400024D9F582E43401F583E004F87E007401A3
:10395000088005C333CE33CED8F9FFED75F00EA441
:1039600024DAF582E43401F583EEF0A3EFF00D8064
:103970009F22300A5E20005BC20A902E12E0FFA355
:10398000E09001A7CFF0A3EFF0E4FF123E02902EEB
:1039900012E0FEA3E0FF7C007D0A12144A90014D64
:1039A000E02FFF90014CE03EFE90013CE0FBA3E0E5
:1039B000FAA3E0F9EE8FF01215609001A7E0FFA3E3
:1039C000E0902E12CFF0A3EFF09001ED7403F0A37E
:1039D0007420F0229001A77408F0A3E4F0A3743FD0
:1039E000F0A374DFF0E4FDFCF9758A10538AEF0050
:1039F0009001A7E0FEA3E02DF582EE3CF583E49371
:103A0000FF69F90DBD00010CBC37E5BDDFE2900197
:103A1000A9E0FEA3E0F5828E83E493FFE96F7008CE
:103A20009000017403F08005E4900001F0758A10A5
:103A3000538AEF0022E4FEEEC39407748094805012
:103A400039EE75F003A42417F582E4342EF583E5EE
:103A5000822FF582E43583F583E493FDEE75F00360
:103A6000A42416F582E4342EF583E4932420F58211
:103A7000E4342EF583EDF00E80BDEF701090014C14
:103A8000E07002A3E07006902E217412F022E49000
:103A900001A7F0A3F0758A10538AEF00122DE47588
:103AA000EA81E4F5F6F5F475F308F5F275EB070035
:103AB000E5EC30E7FBAFF3EFFEADF2EDFF9001393F
:103AC000E0FBA3E0FAA3E0F9EE8FF0121560E4F555
:103AD000EC75EB30758A10538AEF0022900108E0F4
:103AE000FBA3E0FAA3E0F974FF75F0F91215289032
:103AF0000197E02407F0900196E03400F0900194E3
:103B0000E0FEA3E0FFC394E8EE9403501BEF94079C
:103B1000EE9400400CE024F9F0900194E034FFF0C2
:103B200022E4900194F0A3F022900108E0FBA3E0CE
:103B3000FAA3E0F9E475F007121528900195E02446
:103B400007F0900194E03400F0900196E0FEA3E0CD
:103B5000FFC3942CEE9401501BEF9407EE940040A9
:103B60000CE024F9F0900196E034FFF022E490019B
:103B700096F0A3F022900036E0FF9000FFE06F6027
:103B80003D900036E0FD9000FFF0900007E09001CE
:103B9000FFF0540FF0ED7E0064207005E0442080BB
:103BA0000CEF64104E700B9001FFE04410F0900099
:103BB00007F0C28A9001EF7403F0A374E8F022903A
:103BC0000025E06410703FF5B2758D20438D2053C1
:103BD0008D7F53A8F7F58BE5DB5404701320091093
:103BE000F58AF586758703000000758601758A10D1
:103BF000758B019001FD7401F09001ED7403F0A349
:103C00007420F0123E42229001A9EFF07E007F1056
:103C1000EEC0E0EFC0E07D00E075F010A42400F9F4
:103C2000740235F0FA7B01D0E0FFD0E0FE121740BD
:103C30009001A9E0C454F0240EF582E43402F58327
:103C4000740BF0A374B8F022E4FFEFC3940B7480FC
:103C50009480502BEF25E02401F582E4342EF58387
:103C6000E493FEEF25E02400F582E4342EF583E4AE
:103C7000932420F582E4342EF583EEF00F80CB9070
:103C80002F56E0902E2BF0229001AF7401F090019E
:103C9000AFE0C394037480948050217F0112368D6D
:103CA000122E2B900102E0FBA3E0FAA3E0F9EE8FC5
:103CB000F01215609001AFE004F080D2E49001F3BF
:103CC000F0A3F022900158E02418FF900157E0344F
:103CD000FCFEC3900166E09F900165E09E50149049
:103CE000016DE07002A3E0701190016D04F0A37407
:103CF000F4F022E490016DF0A3F022EF903E88935F
:103D0000903E8093FE540FFDF87401088002C33387
:103D1000D8FCFDEE54F06008EDF452915293800906
:103D2000ED42ABEDF4528952965389FD22EF903E5D
:103D30008893903E8093FE540FFDF8740108800232
:103D4000C333D8FCFDEE54F06008ED4291ED42889B
:103D50008006ED4289ED4280438902227F011236BE
:103D60008D122E2B900102E0FBA3E0FAA3E0F9EE06
:103D70008FF0121560121F1712176C123360122683
:103D80001D123B75123CC4023972C109C10A4101BE
:103D9000FF004101FE00C103C101C100C102C10514
:103DA000011400C104C106C108C1074100FF10434E
:103DB000021601021900758A10538AEFE4F5867520
:103DC0008F04F5ABF5AC43AC0C7580FF7588FF75BF
:103DD00089FF759104F595F592D28A22900165E0EC
:103DE000FEA3E0FF900163EEF0A3EFF0E4FCFD9092
:103DF00001BE1216D6900167E0FCA3E0FD7F010230
:103E00001B4B9001A9EFF0123CFB9001A9E0FF12BF
:103E10003A359001A9E0903E8893FF122FD8900187
:103E2000A9E0FF023D2DE4F5DA75DA4043DA2075AA
:103E3000D74075D64075DA5843A80275B80475F8AE
:103E40000422E5B254016006E5A85410700F75B263
:103E50009275B6F9E4F5B743B20143A8102278147D
:103E6000E6FF2400F582E4340022EE30E707C3E4E5
:103E70009FFFE49EFE2204001E0014050028001E81
:103E800002030410111500010107000000000000EA
:103E90000000000000000000000000000000000022
:103EA0000000000000000000000000000000000012
:103EB0000000000000000000000000000000000002
:103EC00000000000000000000000000000000000F2
:103ED00000000000000000000000000000000000E2
:103EE00000000000000000000000000000000000D2
:103EF00000000000000000000000000000000000C2
:103F000000000000000000000000000000000000B1
:103F100000000000000000000000000000000000A1
:103F20000000000000000000000000000000000091
:103F30000000000000000000000000000000000081
:103F40000000000000000000000000000000000071
:103F50000000000000000000000000000000000061
:103F60000000000000000000000000000000000051
:103F70000000000000000000000000000000000041
:103F80000000000000000000000000000000000031
:103F90000000000000000000000000000000000021
:103FA0000000000000000000000000000000000011
:103FB0000000000000000000000000000000000001
:103FC00000000000000000000000000000000000F1
:103FD000000000000000000000000000000000C61B
:103FE00000000000000000000000000000000000D1
:103FF00000000000000000000000000000000000C1
:00000001FF
